:020000040000FA
:02000000D32803
:08000800F000030EF100831269
:1000100003130B11813081007C088500F20A7310F4
:10002000861873141328142815281628172818283A
:1000300019281A281B281C28143085007B03031D4F
:1000400048287E0E07397F0203182F28FE1B2C2814
:100050000000061086153228861106143228302832
:10006000061086117E0807397F0203184028FE1902
:100070003D280000061286164328861206164328DD
:10008000412806128612FF0A7F08073A0319FF016A
:10009000FB08031D6328731E6328F808031D5728F7
:1000A0007A08F9000930F80055280611632803146E
:1000B000F90C03185E280000061160280615602858
:1000C000F80303197312F40803197C287403031945
:1000D000F5017318F50AF40A741E81280130F40042
:1000E000F8307507F60C031881287608F700F31826
:1000F0007315F314F401812873188128FF30F6007A
:10010000F40AFB0A0F307B060319FB017B08820708
:1001100097289728972897289728972897289828E6
:100120009B289D28A528A728AF28B128BF28C32829
:1001300099309F00C3281F15C328FD15C0301E0726
:10014000031CFD1181309F00C3281F15C3287D1596
:10015000C0301E07031C7D1189309F00C3281F1566
:10016000C3287C1AB928FD1480301E07031CFD101B
:10017000C3287D1480301E07031C7D10C328103057
:100180007C1A0430FC00710E8300F00E700E090022
:10019000731AC828FA0073160800F31CCD287708D4
:1001A000F31073110800143085000430860081308C
:1001B0009F00831604309F00EB308500C23086001C
:1001C000083081008312F4010430FC00FF30FD0090
:1001D000F600F301F801FF01FE01F201FB018101CC
:1001E0000B118B168B177D08C820CD20FE00F3283D
:02400E00621A34
:00000001FF
